S01800005A656974736368616C74756E675F56362E73726563BC
S11300000C9435000C9452000C9452000C94520041
S11300100C9452000C9452000C9452000C94520014
S11300200C9452000C9452000C9452000C94520004
S11300300C9452000C9452000C9452000C945200F4
S11300400C9452000C9452000C9452000C945200E4
S11300500C9452000C9452000C9452000C945200D4
S11300600C9452000C945200950011241FBECFEF43
S1130070D4E0DEBFCDBF21E0A0E0B1E001C01D921D
S1130080A030B207E1F710E0CAE6D0E004C022973E
S1130090FE010E949D00C836D107C9F70E94600086
S11300A00C94A1000C9400005E98569A08955E9AF0
S11300B0569A08955F98579A08955F9A579A0895A3
S11300C00E9457000E945A002FEF84E39CE02150C5
S11300D080409040E1F700C000000E9457000E9459
S11300E05D002FEF84E39CE0215080409040E1F7D5
S11300F000C000000E9454000E945D002FEF84E3C2
S11301009CE0215080409040E1F700C000000E9434
S113011054000E945A002FEF84E39CE02150804059
S11301209040E1F700C00000CBCF579A569A0E9446
S113013054000C945A00EE0FFF1F0590F491E02D2B
S10901400994F894FFCFBE
S9030000FC
